:100000000C9472000C949A000C949A000C949A0030
:100010000C949A000C949A000C949A000C949A00F8
:100020000C949A000C949A000C949A000C949A00E8
:100030000C949A000C949A000C949A000C949A00D8
:100040000C9464050C949A000C9432050C940C05E5
:100050000C949A000C949A000C949A000C949A00B8
:100060000C949A000C949A000000000024002700D1
:100070002A0000000000250028002B0000000008D6
:10008000000201000003040700000000000000005F
:10009000C2BA432000252054656D70657261747585
:1000A00072613A200048756D656461643A20000011
:1000B00000000023002600290004040404040404B2
:1000C0000402020202020203030303030301020407
:1000D00008102040800102040810200102040810CA
:1000E0002000AE0511241FBECFEFD8E0DEBFCDBF8C
:1000F00011E0A0E0B1E0E2E6F4E102C005900D926B
:10010000A832B107D9F721E0A8E2B1E001C01D9201
:10011000A13EB207E1F710E0C2E7D0E004C02197AA
:10012000FE010E94290AC137D107C9F70E94FB05C9
:100130000C942F0A0C940000CF92DF92EF92FF9262
:10014000CF93DF93B091D501A0E08111AB2F8091C7
:10015000D60190E0880F991FAC0141555F4FC090C8
:10016000DB01D090DC01E090DD01F090DE0130E0B9
:1001700020E0FA01C591D491E881B90190E080E0D6
:10018000EB23EA130AC02F5F3F4F6C157D058E05E8
:100190009F0578F36FEF7FEFCB01DF91CF91FF9059
:1001A000EF90DF90CF900895AF92BF92CF92DF9201
:1001B000EF92FF920F931F93CF93DF936C017B011C
:1001C0008B01040F151FEB015E01AE18BF08C017AD
:1001D000D10759F06991D601ED91FC910190F08120
:1001E000E02DC6010995892B79F7C501DF91CF91E3
:1001F0001F910F91FF90EF90DF90CF90BF90AF9045
:100200000895FC01538D448D252F30E0842F90E01C
:10021000821B930B541710F0CF9608950197089501
:10022000FC01918D828D981761F0A28DAE0FBF2FCA
:10023000B11D5D968C91928D9F5F9F73928F90E020
:1002400008958FEF9FEF0895FC01918D828D98178F
:1002500031F0828DE80FF11D858D90E008958FEFCC
:100260009FEF0895FC01918D228D892F90E0805C95
:100270009F4F821B91098F739927089581E391E025
:100280000E94320121E0892B09F420E0822F089599
:1002900080E090E0892B29F00E943E0181110C94AE
:1002A00000000895FC01A48DA80FB92FB11DA35A19
:1002B000BF4F2C91848D90E001968F739927848F86
:1002C000A689B7892C93A089B1898C9183708064A9
:1002D0008C93938D848D981306C00288F389E02D4A
:1002E00080818F7D80830895EF92FF920F931F93FB
:1002F000CF93DF93EC0181E0888F9B8D8C8D9813D9
:100300001AC0E889F989808185FF15C09FB7F894E4
:10031000EE89FF896083E889F98980818370806430
:1003200080839FBF81E090E0DF91CF911F910F917B
:10033000FF90EF900895F62E0B8D10E00F5F1F4F8A
:100340000F731127E02E8C8D8E110CC00FB607FC99
:10035000FACFE889F989808185FFF5CFCE010E9427
:100360005201F1CFEB8DEC0FFD2FF11DE35AFF4F42
:10037000F0829FB7F8940B8FEA89FB8980818062B5
:10038000CFCF0F931F93CF93DF938C01D0E0C0E0CA
:10039000F801EC0FFD1F6491662341F081E391E0C9
:1003A0000E947401892B11F02196F2CFCE01DF91CA
:1003B000CF911F910F910895CF93DF93EC01888D1A
:1003C0008823B9F0AA89BB89E889F9898C9185FDD0
:1003D00003C0808186FD0DC00FB607FCF7CF8C915E
:1003E00085FFF2CF808185FFEDCFCE010E945201C3
:1003F000E9CFDF91CF91089590E0FC01E458FF4FE1
:100400002491FC01E353FF4F3491FC01E754FF4F6B
:10041000E491EE23C9F0222339F0233001F1A8F44E
:10042000213019F1223029F1F0E0EE0FFF1FEE58D4
:10043000FF4FA591B4918FB7F894EC91611126C04C
:1004400030953E233C938FBF08952730A9F0283084
:10045000C9F0243049F7809180008F7D03C08091DE
:1004600080008F7780938000DFCF84B58F7784BD45
:10047000DBCF84B58F7DFBCF8091B0008F778093E9
:10048000B000D2CF8091B0008F7DF9CF3E2BDACF74
:10049000CF93DF9390E0FC01E353FF4F2491875407
:1004A0009F4FFC0184918823D1F090E0880F991F21
:1004B000FC01E859FF4FA591B491FC01EE58FF4FA4
:1004C000C591D491623071F49FB7F8943C91822F1A
:1004D000809583238C93E8812E2B28839FBFDF9107
:1004E000CF9108958FB7F894EC912E2B2C938FBF5A
:1004F000F6CF3FB7F8948091290190912A01A091FD
:100500002B01B0912C0126B5A89B05C02F3F19F0F7
:100510000196A11DB11D3FBFBA2FA92F982F882783
:10052000BC01CD01620F711D811D911D42E0660F5E
:10053000771F881F991F4A95D1F708958F929F9230
:10054000AF92BF92CF92DF92EF92FF924B015C018C
:100550000E9479026B017C010E9479026C197D096D
:100560008E099F09683E734081059105A8F321E03B
:10057000821A9108A108B10888EEC80E83E0D81E3F
:10058000E11CF11C81149104A104B10429F7FF902E
:10059000EF90DF90CF90BF90AF909F908F90089595
:1005A000CF92DF92EF92FF920F931F93CF93DF933F
:1005B000CDB7DEB7C054D1400FB6F894DEBF0FBE42
:1005C000CDBF2FB7F89480912D0190912E01A0916D
:1005D0002F01B09130012FBF4091D7015091D80128
:1005E0006091D9017091DA018C019D01041B150BFA
:1005F000260B370BB901A801403D57406105710535
:1006000090F48091DF01C05CDE4F0FB6F894DEBF3E
:100610000FBECDBFDF91CF911F910F91FF90EF9053
:10062000DF90CF9008958093D7019093D801A09345
:10063000D901B093DA011092D2011092D101109237
:10064000D0011092CF011092CE0162E08091D301CF
:100650000E94480261E070E080E090E00E949E020B
:1006600061E08091D3010E94480260E08091D30153
:100670000E94FC018091D4018551823020F58BE2EB
:1006800091E10197F1F762E08091D3010E94480265
:100690008091E00190E08230910538F0880F991F39
:1006A000880F991F05970197F1F7F89480E00E9451
:1006B0009C006F3F7F4F8F4F9F4F61F41092DF017F
:1006C000789480E0A0CF64E170E080E090E00E9448
:1006D0009E02D9CF81E00E949C006F3F7F4F8F4FD9
:1006E0009F4F61F38E010F5F1F4F6E018FEBC81A92
:1006F0008EEFD80A780180E00E949C00F7016083A9
:1007000071838283938381E00E949C00F70164835C
:10071000758386839783F8E0EF0EF11CEC14FD04DB
:1007200051F7789430E020E0F801C080D180E28079
:10073000F3804481558166817781FFEFCF16DF0614
:10074000EF06FF0631F04F3F8FEF58076807780735
:1007500019F41092DF01B5CFF90183E0F595E79523
:100760008A95E1F7E253FE4F8081880FC416D506C3
:10077000E606F70610F180832F5F3F4F085F1F4F9B
:100780002832310589F64091D2012091CE01809125
:10079000CF01280F3327331F8091D001280F311D3F
:1007A0008091D101820F932F911D99274817190627
:1007B00081F681E08093DF0126CF8160DCCFFC01F0
:1007C00001900020E9F73197AF01481B590BBC019C
:1007D00081E391E00C94D4008F929F92AF92BF92EC
:1007E0000F931F93CF93DF93CDB7DEB7A1970FB6CB
:1007F000F894DEBF0FBECDBF19A2423008F44AE024
:100800008E010F5D1F4F842E912CB12CA12CA501C0
:1008100094010E94070AE62FB901CA01EA30F4F4F4
:10082000E05DD801EE938D01232B242B252B79F746
:1008300090E080E0109719F0CD010E94DF03A196AF
:100840000FB6F894DEBF0FBECDBFDF91CF911F91E1
:100850000F91BF90AF909F908F900895E95CE1CF8A
:100860004F925F926F927F928F929F92AF92BF92C0
:10087000CF92DF92EF92FF920F931F93CF936B0172
:100880007C01742EAC019B010E94020A882399F01E
:1008900082E191E0CF911F910F91FF90EF90DF9057
:1008A000CF90BF90AF909F908F907F906F905F9010
:1008B0004F900C94DF0346015701E894B7F82FEFEF
:1008C0003FEF4FE75FE7C501B4010E94020A8111C3
:1008D0000DC02FEF3FEF4FE75FE7C501B4010E9466
:1008E000380818161CF486E191E0D4CF2FEF3FEFC3
:1008F0004FE75FE4C701B6010E94900918161CF487
:100900008AE191E0C7CF2FEF3FEF4FE75FECC701E0
:10091000B6010E94380887FDF3CF20E030E0A9013E
:10092000C701B6010E94380810E000E087FF0AC046
:100930006DE281E391E00E9474018C01F7FAF0947A
:10094000F7F8F094C0E060E070E080E09FE37C1690
:1009500041F020E030E040E251E40E943D08CF5FEA
:10096000F6CFA70196010E94CC072B013C010E9403
:10097000AF084B015C014AE00E94EC037C01E00EF1
:10098000F11ECC23C1F1C501B4010E94DE089B0118
:10099000AC01C301B2010E94CB074B015C016EE2C6
:1009A00081E391E00E947401E80EF91EC15018F134
:1009B00020E030E040E251E4C501B4010E94950915
:1009C0002B013C010E94AF084B01B12CA12C4AE045
:1009D000C501B4010E94EC03E80EF91EC501B40183
:1009E0000E94DE089B01AC01C301B2010E94CB074B
:1009F0004B015C01DBCFC701CF911F910F91FF909D
:100A0000EF90DF90CF90BF90AF909F908F907F90AE
:100A10006F905F904F9008951F920F920FB60F92B4
:100A200011242F933F934F935F936F937F938F93F3
:100A30009F93AF93BF93EF93FF9381E391E00E9465
:100A40005201FF91EF91BF91AF919F918F917F9153
:100A50006F915F914F913F912F910F900FBE0F902B
:100A60001F9018951F920F920FB60F9211242F937B
:100A70008F939F93EF93FF93E0914101F091420197
:100A80008081E0914701F091480182FD1BC0908177
:100A900080914A018F5F8F7320914B01821741F043
:100AA000E0914A01F0E0EF5CFE4F958F80934A01A0
:100AB000FF91EF919F918F912F910F900FBE0F900B
:100AC0001F9018958081F4CF1F920F920FB60F924E
:100AD00011242F933F938F939F93AF93BF93809154
:100AE0002D0190912E01A0912F01B09130013091F4
:100AF000280123E0230F2D3758F50196A11DB11DC4
:100B00002093280180932D0190932E01A0932F0113
:100B1000B09330018091290190912A01A0912B017D
:100B2000B0912C010196A11DB11D809329019093D4
:100B30002A01A0932B01B0932C01BF91AF919F91FB
:100B40008F913F912F910F900FBE0F901F9018958E
:100B500026E8230F0296A11DB11DD2CFE1E3F1E0FB
:100B60001382128288EE93E0A0E0B0E08483958344
:100B7000A683B78384E091E09183808385EC90E045
:100B80009587848784EC90E09787868780EC90E057
:100B9000918B808B81EC90E0938B828B82EC90E048
:100BA000958B848B86EC90E0978B868B118E128EC2
:100BB000138E148EAEECB1E082E015968C931597EF
:100BC0008BE016968C931697EFECF0E0E491179675
:100BD000EC931797EBEBF0E0E4911896EC931897F1
:100BE00040E85EE360E070E01D964D935D936D9389
:100BF0007C9350970895789484B5826084BD84B5C1
:100C0000816084BD85B5826085BD85B5816085BD07
:100C100080916E00816080936E00109281008091BF
:100C20008100826080938100809181008160809347
:100C30008100809180008160809380008091B1006C
:100C400084608093B1008091B00081608093B00097
:100C500080917A00846080937A0080917A0082602B
:100C600080937A0080917A00816080937A008091ED
:100C70007A00806880937A001092C10061E087E07A
:100C80000E94480261E085E00E94480261E086E03F
:100C90000E944802E0914101F091420182E080838C
:100CA000E0913D01F0913E011082E0913F01F09111
:100CB00040018FEC808310924901E0914501F09151
:100CC000460186E08083E0914301F09144018081F8
:100CD00080618083E0914301F091440180818860CC
:100CE0008083E0914301F09144018081806880839A
:100CF000E0914301F091440180818F7D808362E027
:100D00008091D3010E9448022FB7F89480912D0161
:100D100090912E01A0912F01B09130012FBF805DE5
:100D20009740A109B1098093D7019093D801A0936E
:100D3000D901B093DA0187E38093E001C0E0D0E00D
:100D400060ED77E080E090E00E949E020E94D00279
:100D5000882349F08091D4018B3028F08D3050F0F9
:100D600085518230C0F1812C912C20ECA22E2FE7EE
:100D7000B22E1EC06091CF0170E090E080E00E9432
:100D8000E0082DEC3CEC4CEC5DE30E9495096B0116
:100D90007C016091CE0170E090E080E00E94E0086C
:100DA0009B01AC01C701B6010E94CC074B015C015D
:100DB0000E94D002882341F08091D4018C3009F444
:100DC0009AC0D8F48B3091F1C12CD12C80ECE82E54
:100DD0008FE7F82E55C06091CE017091CF01762734
:100DE0006727762790E080E00E94DE082DEC3CEC3F
:100DF0004CEC5DE30E949509D9CF8551823020F7F4
:100E00001091D001612F70E0762F662766277F77DB
:100E10008091D101682B90E080E00E94DE082DECEB
:100E20003CEC4CEC5DE30E94950981C06091D001DF
:100E300070E090E080E00E94DE086B017C01109180
:100E4000D10117FF0AC0AC019B0160E070E080E8AF
:100E50009FEB0E94CB076B017C011F70612F70E03C
:100E600090E080E00E94E0082DEC3CEC4CEC5DE36F
:100E70000E949509A70196010E94CC076B017C0195
:100E800085EA90E00E94C10142E0C501B4010E94E0
:100E9000300485E990E00E94C10142E0C701B6013B
:100EA0000E94300480E990E00E94C10120E030E01F
:100EB00040EE51E4C701B6010E94900987FD40C091
:100EC00061E087E00E94FC0160E085E00E94FC0197
:100ED00060E086E00E94FC018EE191E00E94DF0369
:100EE000209709F42DCF0E943E01882309F428CFD2
:100EF0000E94000025CF1091D001612F70E090E09A
:100F000080E00E94DE086B017C016091D1016F706E
:100F100070E090E080E00E94E0082DEC3CEC4CECAE
:100F20005DE30E949509A70196010E94CC076B0121
:100F30007C0117FFA5CFF7FAF094F7F8F094A0CF53
:100F400020E030E040EA51E4C701B6010E94900978
:100F500087FD17C020E030E040ED51E4C701B60145
:100F60000E94380818166CF060E087E00E94FC01CF
:100F700061E085E00E94FC0160E086E00E94FC01E7
:100F8000AFCF60E087E00E94FC0160E085E00E9456
:100F9000FC0161E0F2CF5058BB27AA270E94E3076B
:100FA0000C9456090E94480938F00E944F0920F01D
:100FB00039F49F3F19F426F40C9445090EF4E0959A
:100FC000E7FB0C943F09E92F0E94670958F3BA1711
:100FD000620773078407950720F079F4A6F50C944F
:100FE00089090EF4E0950B2EBA2FA02D0B01B90143
:100FF00090010C01CA01A0011124FF27591B99F08F
:10100000593F50F4503E68F11A16F040A22F232F9A
:10101000342F4427585FF3CF469537952795A795EA
:10102000F0405395C9F77EF41F16BA0B620B730B91
:10103000840BBAF09150A1F0FF0FBB1F661F771F02
:10104000881FC2F70EC0BA0F621F731F841F48F4B7
:10105000879577956795B795F7959E3F08F0B0CF40
:101060009395880F08F09927EE0F97958795089527
:101070000E941B0908F481E008950E9451080C9415
:1010800056090E944F0958F00E94480940F029F47F
:101090005F3F29F00C943F0951110C948A090C947C
:1010A00045090E94670968F39923B1F3552391F329
:1010B000951B550BBB27AA2762177307840738F0C7
:1010C0009F5F5F4F220F331F441FAA1FA9F335D024
:1010D0000E2E3AF0E0E832D091505040E695001CD8
:1010E000CAF72BD0FE2F29D0660F771F881FBB1F92
:1010F000261737074807AB07B0E809F0BB0B802D70
:10110000BF01FF2793585F4F3AF09E3F510578F09B
:101110000C943F090C948A095F3FE4F3983ED4F3A2
:10112000869577956795B795F7959F5FC9F7880F6F
:10113000911D9695879597F90895E1E0660F771FC1
:10114000881FBB1F621773078407BA0720F0621B52
:10115000730B840BBA0BEE1F88F7E09508950E947D
:101160006F0988F09F5798F0B92F9927B751B0F0C1
:10117000E1F0660F771F881F991F1AF0BA95C9F71B
:1011800014C0B13091F00E948909B1E008950C9427
:101190008909672F782F8827B85F39F0B93FCCF3DA
:1011A000869577956795B395D9F73EF49095809598
:1011B000709561957F4F8F4F9F4F0895E89409C0B8
:1011C00097FB3EF490958095709561957F4F8F4F7A
:1011D0009F4F9923A9F0F92F96E9BB279395F69590
:1011E000879577956795B795F111F8CFFAF4BB0F0E
:1011F00011F460FF1BC06F5F7F4F8F4F9F4F16C072
:10120000882311F096E911C0772321F09EE8872FFB
:10121000762F05C0662371F096E8862F70E060E0B7
:101220002AF09A95660F771F881FDAF7880F969530
:10123000879597F90895990F0008550FAA0BE0E8D4
:10124000FEEF16161706E807F907C0F01216130688
:10125000E407F50798F0621B730B840B950B39F4C8
:101260000A2661F0232B242B252B21F408950A262E
:1012700009F4A140A6958FEF811D811D089597F96E
:101280009F6780E870E060E008959FEF80EC08952C
:1012900000240A9416161706180609060895002455
:1012A0000A9412161306140605060895092E0394CF
:1012B000000C11F4882352F0BB0F40F4BF2B11F443
:1012C00060FF04C06F5F7F4F8F4F9F4F089557FDA2
:1012D0009058440F551F59F05F3F71F04795880FA4
:1012E00097FB991F61F09F3F79F08795089512163B
:1012F00013061406551FF2CF4695F1DF08C01616E7
:1013000017061806991FF1CF869571056105089497
:101310000895E894BB2766277727CB0197F90895AE
:101320000E941B0908F48FEF08950E94A8090C94ED
:1013300056090E94480938F00E944F0920F0952371
:1013400011F00C943F090C94450911240C948A095E
:101350000E94670970F3959FC1F3950F50E0551FE8
:10136000629FF001729FBB27F00DB11D639FAA27FA
:10137000F00DB11DAA1F649F6627B00DA11D661F49
:10138000829F2227B00DA11D621F739FB00DA11D6A
:10139000621F839FA00D611D221F749F3327A00D24
:1013A000611D231F849F600D211D822F762F6A2FC0
:1013B00011249F5750409AF0F1F088234AF0EE0F25
:1013C000FF1FBB1F661F771F881F91505040A9F752
:1013D0009E3F510580F00C943F090C948A095F3FB1
:1013E000E4F3983ED4F3869577956795B795F7958E
:1013F000E7959F5FC1F7FE2B880F911D9695879506
:1014000097F908950E941B09880B990B0895A1E292
:101410001A2EAA1BBB1BFD010DC0AA1FBB1FEE1F6E
:10142000FF1FA217B307E407F50720F0A21BB30BB9
:10143000E40BF50B661F771F881F991F1A9469F735
:1014400060957095809590959B01AC01BD01CF0191
:101450000895EE0FFF1F0590F491E02D0994F89484
:02146000FFCFBC
:10146200000000007401D4000101DC01320110010E
:1014720024016E616E00696E66006F7666005472BA
:081482006F6C61736F3A2000EA
:00000001FF
